:020000040800F2
:1050000034483349016034494160344901613449CD
:1050100081603449C1603449416134498161344916
:10502000016234494162344981623449C162344980
:105030000163344941633449C1633449816334496C
:10504000C16134494164344981643449016434495B
:10505000C164344901653449416534498165344945
:10506000C165344901663449816634494166344931
:10507000C16634490167344941673449C1673449DD
:105080008167803033490160334941603349816031
:105090003349C16033490161334901623349416297
:1050A00033494161334981613349C1613349016306
:1050B000334981623349C162334941633349816372
:1050C000704710B500F064FB00F02EFC002010BD0E
:1050D00017620008740500200F760008519500083B
:1050E00087760008518300086D6700086B7100081F
:1050F000CD510008436500083D6700085D99000830
:10510000D75E0008AF79000865520008E351000837
:105110005F550008C15B0008677B000899750008AF
:105120004B7500085554000805550008876D0008A8
:10513000EF750008A9560008455F00087D5D00086E
:1051400093560008CF970008975E000803560008A2
:1051500047630008497600083B7100080384000893
:1051600055840008AB84000841950008755E00086E
:10517000C3730008A19400085D5D0008078600085D
:105180009D740008E3940008D7840008FD99000886
:10519000302802D94FF0FF307047A74A202802EB91
:1051A000800202D922F8821C0EE0102806D952F89B
:1051B000440D00F0FF1040EA012004E052F8040D15
:1051C0009E4B184008431060002070479A4A002008
:1051D0006FF07F4142F82010401CC0B20F28F9D96F
:1051E0007047F0B5401EC4B2601E0D46302802D391
:1051F0004FF0FF30F0BD924F0A26A7F1240C95FB2B
:10520000F6F006FB105095FBF6F5C1B2385D641E52
:10521000E4B21CF80110FFF7BBFF002DEFDC00200B
:10522000F0BD8749A0F141023E390144192A02D854
:1052300011F9410C7047A0F16102192A02D811F945
:10524000610C7047A0F13001092901D848B27047BC
:105250002D2803D02E2803D023207047212070470B
:1052600022207047F0B5764F00250E460446243FB5
:10527000DFF8CCC112E0FFF7D4FFC0B2395C0CEB11
:10528000040010F8010CFFF783FF641CE4B2302C1B
:1052900002D94FF0FF30F0BD6D1CEDB2705D0028FB
:1052A000E9D1F0BD70B5044663480D464030FEF7C5
:1052B0005DFE2846FEF77EFE6149C0B246390123F5
:1052C00088704D7900222DB12044401EC8704A706C
:1052D0000B7103E0CC70401E48700A714A718A71EC
:1052E000CB710B7070BD2DE9F0470346FFF76EFFE1
:1052F000DFF84CA1DFF84C91AAF1240AF3B34FF088
:10530000000800252FE0002425E04D4FD4461AF870
:105310000510385DFFF73CFF3E191CF8051016F824
:10532000100FFFF735FF1CF80510307CFFF730FF3A
:10533000C82004F0B5F8385DFF21FFF729FF307869
:10534000FF21FFF725FF307CFF21FFF721FF641CC1
:10535000E4B20F2C03D899F800000028D5D06D1CBA
:10536000EDB21E2D03D899F800100029CBD008F11A
:10537000010000F0FF08B8F10F0F00E001E0C0D914
:105380002EE0002556464FF4C8784F46002420E012
:105390004FF0010C315D6046FFF7FAFE0CF1010C95
:1053A0000CF0FF0CBCF1300FF4D9404604F078F853
:1053B0004FF0010CFF216046FFF7EAFE0CF1010CF3
:1053C0000CF0FF0CBCF1300FF4D9641CE4B21D2CBE
:1053D00002D838780028DBD06D1CEDB2282DD5D945
:1053E00099F8000010B9184901200860FFF7EEFE97
:1053F00016490120FFF736FFBDE8F04714490720A2
:1054000030E7704710B50C4C0021403400F00F021B
:10541000C1F105030009E254092A01D9413200E033
:105420003032491CC9B2E2540629EFD30020A071E2
:105430000148403010BD0000BC0A002000FFFF0002
:10544000530200202C09002030090020BC08002055
:10545000D808002070B5AD4D420730D50C0901F0D9
:105460000F01820702D5285D484005E0C00705D03E
:10547000285DC1F10F010840285500E02955A44ED0
:105480003088C00705D03188C807FCD1052004F05A
:1054900028F8A048C1684FF60F7211402A5D41EA12
:1054A0000211C1609C480168C1F30A0141EA04315C
:1054B000016001213046FBF7AFFA002070BD3129B1
:1054C00002D94FF0FF3070BD4A1ED31702EB937222
:1054D000C2F3870422F00302491E8A1A0121914077
:1054E000C9B2C20702D0285D084307E08007285DE3
:1054F00001D5484002E0C1F10F010840285500F0F5
:105500000F00B9E72DE9F0478448804EDFF80082AC
:10551000DFF80092804F056800244FF60F7A315D66
:1055200015F8010B0143315540460288D207FCD1E2
:10553000D9F80C2002EA0A0242EA0111C9F80C105B
:105540003968C1F30A0141EA043139600121FBF7EE
:1055500063FA641CE4B20C2CE1D3BDE8F0872DE9BA
:10556000F0476E48694EDFF8A881DFF8A8916A4FCE
:10557000056800244FF60F7A15F8010B315DC0F174
:105580000F000140315540460288D207FCD1D9F8BE
:105590000C3003EA0A0343EA0111C9F80C10396818
:1055A000C1F30A0141EA043139600121FBF734FA01
:1055B000641CE4B20C2CDFD3CFE7411ECA1701EB09
:1055C000927230B5554901240B6803EBA20209E041
:1055D000312814D0401CC0B2411ECA1701EB927191
:1055E00003EBA102411ECD1701EB957525F00305D4
:1055F0001278491B04FA01F10A42E9D030BD0420B7
:10560000EAE72DE9F0410024444E14270B20FEF771
:105610008AF8401C05B21020FEF785F83168495D14
:10562000014041EA0510C1B20420FFF713FF142026
:1056300003F057FFB4FBF7F007FB104008B9FFF782
:1056400061FF641CC82CE1D3BDE8F0812DE9F0476F
:105650000024DFF8B8902E4F2E4D2F4EA0464FF667
:105660000F7A09F8048038460188C907FCD1E96837
:1056700001EA0A01E9603168C1F30A0141EA043133
:1056800031600121FBF7C8F9641CE4B20C2CE8D3AB
:1056900063E71E49002001F10C020B5C1354401C0F
:1056A000C0B20C28F9D3704770B5184D00240C35E2
:1056B000285D40EA0410C1B20420FFF7CBFE641C51
:1056C000E4B20C2CF4D370BD70B5154C4FF4967049
:1056D0004FF4FA76134D20600FE0FFF713FF3046CA
:1056E00003F0DEFEFFF73BFF287810B9304603F0E9
:1056F000D7FE2168491E216002D028780028ECD00E
:105700002878002801D10120206070BD150B0020F1
:1057100000040040001001400C0C01409C080020D7
:10572000300900202C09002070B5D34D0420D34946
:10573000E87002200870D24800240470D148047038
:1057400003F06BF9D149D0480860D1490860D148CD
:105750002C70AC70047070BD10B5CE480024CEA182
:1057600004700120FFF77EFD03F008FBFDF7FDFC50
:1057700020B1CBA10120FFF775FD01E0FFF726FD69
:10578000C948BE49046002200870C848047010BDB2
:1057900070B5C748016841F4E0210160C5484FF485
:1057A0007A76C5490660C8200870C4490F200025D4
:1057B0000870B24902200870C1480570FDF737FD36
:1057C000FDF7B2FDFDF77FFDFAF7C0FEFDF714FD12
:1057D000FDF7BEFEFDF707FEFDF72DFEFDF75AFEB5
:1057E000FDF783FEB7480124C0F8AC41FFF708FC81
:1057F000FFF72CFF00F00BFAFFF7E8FCB249C1F805
:105800009441C1F8984100F066FBFDF7FAFCFBF704
:1058100086FE30B9FBF7DDFC0120FBF71AFEFBF733
:10582000DEFCFDF78AFF03F01EFF03F078FEFFF7B2
:105830007BFFFDF7B4FD0020FDF780FC9548007864
:10584000401E0B2802D30020FFF786FFFDF701FC66
:1058500030B19EA10120FFF705FD304603F041FE67
:105860000020FDF776FC904C9C4E2168884201D1C7
:10587000307878B39AA10120FFF7F4FC9AA10720B1
:10588000FFF7F0FC03F013F835700020FDF761FC22
:105890002060FDF76AFC4FF4487003F022FE002000
:1058A000FDF757FC2168884212D091A10120FFF733
:1058B000D9FC91A10720FFF7D5FC4FF4C87003F085
:1058C00010FEFDF73AFF642003F00BFEFDF735FFF5
:1058D000FFF77CFC8A48008881B28A48007804F08F
:1058E0008DF88948008881B28848007804F086F8ED
:1058F00087480068804701F0F0FB86A10120FFF790
:10590000B1FC86490920FFF7ADFC85A11120FFF706
:10591000A9FC594881681920FFF7A4FCBDE8704034
:105920004FF4FA6003F0DDBDDFF8FCB17F4F574E56
:10593000DFF84891DFF8F8A14FF000084E4CE0780E
:10594000012801D0022819D12079032814D37948DD
:105950006C4900680978007A88420DD07649FDF7D5
:10596000B5FE76A17A48FEF701FB73497848FEF749
:1059700040FB7748FEF77FFA03F06DFF444D316836
:105980002868884256D000F0C1FA6070FF2851D0D4
:10599000217979B100F0AFFA6749FDF797FE6DA163
:1059A0006B48FEF7E3FA64496948FEF722FB684852
:1059B000FEF761FA6078A0F17001072901D8012192
:1059C00000E000218BF8001099F80020022A03D093
:1059D00029B102F046FF1DE00029FAD11AE000F0DB
:1059E00081FA61490968884700280BDA6178FF2944
:1059F00008D05E48426842F47F4242601620FFF7BA
:105A0000F0FB05E02079012802D159A0FEF733FA16
:105A10008AF80080387850B95F48007803F061FD5B
:105A200028683168884202D0607800F08BFA87F8E5
:105A30000080A4E799F8000001280BD19AF8001023
:105A400050462D2906D380F80080207910B153A04C
:105A5000FEF711FA574C207848B1574D28780128A5
:105A600005D1FEF77FF985F8008084F8008053485F
:105A70000068804762E70000CC030020DD060020BC
:105A8000510300202C090020930B002074060020F5
:105A90007006002048040020202067616D6500002A
:105AA000206572726F720000B00400209E06002014
:105AB00024ED00E0780400202D04002042040020A2
:105AC0008B0800200080214200002342736574751A
:105AD0007020206572726F72200000003804002070
:105AE00020726573657400006E7672616D2000002F
:105AF000206E7672616D000073686F742020000064
:105B00007C0400207407002080040020EC070020A3
:105B10008C02002020702D7265760000DE060020C9
:105B200020672D72657600009A060020A2060020EC
:105B300005090020340900202D0B00204576656EF4
:105B4000742074726967676572202D200000000060
:105B5000230C002053776974636820436C6F73656E
:105B600064202D200000000084020020BC0A0020D8
:105B7000537769746368206E6F742070726F6772F8
:105B8000616D6D656420666F72207468697320674B
:105B9000616D653F213F0000340800205761746348
:105BA00068646F672042616C6C2053656172636842
:105BB0002E0000000409002000000020C002002088
:105BC00030B40346092904D9002B1ED0B1F5007F5B
:105BD0001BD25A480288D207FCD1594ADC0709D0A7
:105BE000146884EAC1141460022B0AD230BC01216B
:105BF000FAF712BF0124891D04FA01F114684C4020
:105C0000F1E7504A10884840108030BC70474C483B
:105C100001684FF6807211430160704710B5044669
:105C200003F014F808B1012010BD21462E20FFF723
:105C3000D8FA21460220FFF70DFC4FF4967003F0CE
:105C400050FC21460220FFF705FC4FF4FA7003F0E8
:105C500048FC002010BD2DE9F04101210026084636
:105C6000FFF7F8FB012455E037A12F20FFF7FAFAE0
:105C70000025364FDFF8D8800AE03868405DFFF72E
:105C8000CDFF02F0E3FF38B900F025F96D1CEDB24D
:105C900098F800008542F0D32EA12F20FFF7E2FAFA
:105CA0002CA12D20FFF7DEFA02F0D0FFB0BB0125BA
:105CB0004FF4FA674FF4487823E029462E20FFF787
:105CC00090FA29460020FFF77BFF0EB1384600E02E
:105CD000404603F006FC00F02BF9742801D126B1F0
:105CE000002602F0B3FF88B901E00126F9E700F0D1
:105CF000F2F816B1641CE4B201E06D1CEDB2092D9E
:105D000004D802F0A3FF08B9142CD6D3641CE4B263
:105D1000142C03D802F09AFF0028A5D002F096FFB9
:105D200010B90D490120086001210020FFF792FB06
:105D3000BDE8F04107A12D20FFF794BA000800400C
:105D40000C180140300600204C530000A008002031
:105D50008B080020202000003009002010B50F29FA
:105D60000BD83B4CE0680843E060282003F0B9FB07
:105D7000E0684FF6F0710840E06010BD70B5054670
:105D80000C46052902D13348007818B9324800780A
:105D9000002818D03148007800B102250F2C0ED908
:105DA0000A210120FFF756FB04F00F012846FFF7F8
:105DB000D5FFBDE870400A210020FFF74BBB284605
:105DC000BDE87040CAE770BD2DE9F0470124DFF857
:105DD0009090244FDFF89080254600264FF47A6A91
:105DE00022A12D20FFF73EFA21462E20FFF7F9F9D8
:105DF000012D03D121460020FFF7C0FF504603F0DC
:105E00004FFB99F80000A8B14546386829688842D8
:105E10000ED000F07BF8742803D07028F5D101264D
:105E2000F3E71F2C02D0641CE4B2EEE70124ECE798
:105E3000012501E06D1CEDB226B9142DD0D30C491B
:105E400001200860BDE8F04708A12D20FFF70ABA3D
:105E500000100140390400203A04002032060020DE
:105E60002C0900207006002074060020202000006D
:105E7000300900200A21B0FBF1F201FB1202B0FB55
:105E8000F1F1C44B012088409A5C024201D000200D
:105E900070470120704730B5BE4CBF4B0C3C2246CA
:105EA000A16852684FF0FF35994201D13F3B00E0B5
:105EB0004B1C9A4201D1284630BD08700020A360D7
:105EC00030BDB4480C38D0E90110814201D0012026
:105ED000704700207047B048AE493F380C398860A1
:105EE0004860704700F00F01000900EB800001EBF3
:105EF0004000C0B270470A21B0FBF1F201FB120270
:105F0000B0FBF1F002EB0010C0B27047A14A0C3AAE
:105F1000D2E90110814201D1FF2070479E4B0878E1
:105F2000994202D1A3F13F0100E0491C5160704742
:105F300098490C39D1E90101884201D1FF2070470D
:105F40000078704730B5934C934A0C3CFF2361684E
:105F500009E00D78854200D10B70914202D18E4943
:105F60003F3900E0491CA568A942F2D130BD70B5A7
:105F70008A4C0546207840B1894E3078012804D1FA
:105F8000FDF7F0FE002030702070824C0C3CD4E90C
:105F90000101884208D1284603F082FAD4E90101C0
:105FA000884201D1FF2070BDBDE87040AEE770B5FA
:105FB00000254FF416763046FFF7D9FF04467028C7
:105FC00007D0742C05D06D1CEDB23C2DF3D300200E
:105FD00070BDC820FFF7CBFF702807D0742802D00F
:105FE000702C0BD006E0702C06D003E0702C05D08E
:105FF000742C01D0012070BD022070BD032070BD43
:1060000070B500254FF496763046FFF7B0FF044692
:10601000FF2804D0702C07D0742C05D01CE04A2037
:10602000FFF728FFC0B174244FF4C870FFF79FFF3B
:10603000702807D0742802D0702C0BD006E0702C8A
:1060400006D003E0702C05D0742C01D0012070BD67
:10605000022070BD032070BD6D1CC82DD4DB002054
:1060600070BD10B5FFF7A3FF4E49087010BD10B505
:10607000FFF7C6FF4B49087010BD464A0A210C3A8B
:106080001078B0FBF1F301FB1301052901D0401C8E
:1060900002E04B2802D0401D107070470020FBE743
:1060A0002DE9F047DFF8EC900025A9F10C09DFF8A5
:1060B000F8A03E4EDFF8F8805AE04FF44870FFF742
:1060C00056FF044670280DD0742C06D025B34C46DC
:1060D0002078FFF7CFFE58B10DE00DB1002547E065
:1060E000012545E00020386042E0FFF7C6FFEFE7FA
:1060F00020780028F9D132682EA115209047217808
:1061000029B11620FFF76DF8FFF7B7FF30E0012047
:10611000207028A1162029E0FF2C37DAFFF7E2FED5
:1061200001461620FFF75DF81420FFF720FFA0427C
:106130001ED1214F0124326820A1012090473268EE
:10614000514607209047FA2003F0CBF93868804782
:10615000642003F0C6F9641C042CECDDFFF7BBFEE1
:10616000326818490120904751460720326890470D
:10617000D8F800004746401EC8F80000401C9CD1DB
:106180003268BDE8F04710A1152010470FA1152077
:10619000ECE7000078060020D20B00200409002064
:1061A00000000020BD060020ED080020B005002002
:1061B000300900202000000094050020636C656118
:1061C0006E200000BC080020202000002D2D0000C3
:1061D00070B5F94CF94D20782978884201D300290F
:1061E00018D1632816D2401C207005210220FFF729
:1061F000C5FD287820B920780F2801D90F202070FC
:10620000EF480078002805D02178BDE870403020A4
:10621000FEF7E7BF70BD10B5EA48EB4C007894F884
:106220002610884214D904210120FFF713F9012018
:1062300004F8170FE17B491CE173E4490A68521C1A
:106240000A6060700221BDE810400846FFF796BD65
:1062500010BDD94A1078002809D0401EC1B2D848D4
:1062600011700078002802D03020FEF7BABF7047C6
:1062700070B5D54C0025607E20B1657602210020E6
:10628000FFF7E8F8D248007803F068FBD1480068CF
:10629000804720B14FF4FA6003F023F901E0FEF7E4
:1062A00095FFCB483038007803F058FBE57084F850
:1062B0002650022084F8450001202070E574BDE8D6
:1062C000704000F040B8C448007800280BD0BE4AA7
:1062D000002100EB4000117102F18001C86101F161
:1062E000680003F074BA7047B749002001F18002DA
:1062F00081F8280081F82900106350639063D0630F
:1063000001231064CB76886681F83900C866086777
:1063100081F83A004867886781F83B00C8671060D9
:1063200081F83C00506081F83E30C87081F82B0045
:1063300081F8360081F82600A84B13618875C8756E
:1063400081F84000704770B59C48007818B19A48B1
:10635000007800287DD09C4C0025012694F845103B
:1063600002291BD094F83E00012872D1E07E01285A
:106370006FD12046082990F8360073D0012968D1E2
:10638000E17C002967D0217D002965D0042860D2F6
:1063900004F5A470007803F0E1FA65E08D48A67476
:1063A000006880472178084353D0894825702438F5
:1063B000007803F0D3FA86481830007803F0CEFA5C
:1063C00083486038007803F0C9FA8148543800786F
:1063D00003F0C4FA7E484838007803F0BFFAA57489
:1063E000FEF7F4FE7E48006880477E4800688047DC
:1063F000082084F8450001212E20FEF7F2FEA57149
:106400000B210020FFF726F804210020FFF722F8D7
:1064100001210846FFF71EF80C210020FFF71AF8AB
:1064200002210020FFF716F8FFF75EFF6E480068B4
:106430008047FFF794F86D4800688047FFF74BFDF1
:106440006B4861490068E06660678031E0674860DA
:1064500003E02EE006E027E023E0FFF734FFE574D9
:10646000257506E0042824D2E57404210020FFF7F6
:1064700085FCFFF7EEFE14F8360F5E49401CC0B2F3
:1064800020700A68521C0A60012813D0022814D018
:1064900003284FF0000113D01C20BDE87040FEF728
:1064A000A0BEBDE87040E3E649480C3803F08FF920
:1064B000E67470BD00210620EFE700210C20ECE718
:1064C0001620EAE7434810B50068804700280ED040
:1064D0003D48817C00290AD090F84500022806D169
:1064E00045A10720FEF7BEFEBDE810402BE710BD1A
:1064F00070B5354C04F18000E17811B1C169491ED5
:10650000C161C069012528B1607978B1002060714E
:1065100004210EE094F826004FF0040120B1012080
:10652000FEF798FF257170BD0020F9E76571042121
:106530000120FEF78FFFBDE8704025486C3803F05E
:1065400046B9214A1046117F407F1429084407D3D9
:1065500001D1D07F01E0A0F1150082F82A00704738
:106560000A2905D301D1907FF7E7A0F10B00F4E7EA
:10657000A0F10100F1E710B508210020FFF720FB92
:106580001F480D4A0168491C01600C4910780978C0
:10659000884201D300290DD163280BD2401CC1B21F
:1065A000074811700078002804D0BDE81040302062
:1065B000FEF717BE10BD0000450400204304002074
:1065C00034040020440400209806002068040020C1
:1065D000EC070020A40200202604002040420F0007
:1065E00090020020A0020020B0020020AC02002097
:1065F00084040020580400202020202020200000B7
:1066000070040020FE4810B500780028D2D0FFF7B3
:10661000B2FFBDE810404FF4967002F062BFC9E7C8
:106620002DE9F041F748F84D007840B9F749E86C9A
:10663000884204DD90FBF1F201FB1200E864F44CA7
:10664000E86C2168884224DDF24E307808B1FFF70B
:10665000D9FFF14FE86C396888421CDD2160EF4CAE
:106660002168884214DD307808B1FFF7CBFF20683D
:106670003860EB4FE86C396888420CDD2160FFF729
:10668000C1FF307818B9FFF7BDFFFFF7BBFFE86C1B
:106690003860BDE8F0812060FBE70246491EC8B2C1
:1066A000D949012380310F2A05D0082A16D90E2A8C
:1066B00008D020B113E090B903204B61704702F07D
:1066C000070006E040B9D04890F84500012803D003
:1066D00002204861022070474B6105E010B10022A2
:1066E0004A617047521C4A6101207047CD480068DA
:1066F000004710B5C44CE07800281ED10120E0709E
:1067000094F8260028B904210020FEF7A3FE0020FB
:10671000E075C548007800280FD0E07A08B1607AAB
:1067200001E0617A19B110B9BE4800688047BF48DE
:106730000078BDE8104003F011B93BE7B24810B54E
:10674000014690F82540897801220023012C02D0CF
:1067500019B1426502E039B183704365416DC1648E
:10676000C0E91823C26525E78270F2E7A64890F8D1
:106770002510012901D0C16C01E0816DC164416522
:1067800001211022C0E91821C1657047082805D9E8
:106790000E2801D2022070470F2801D00120704737
:1067A000032070472DE9F047974D0024012785F815
:1067B0002540102085F83770DFF87482DFF8749276
:1067C00085F838000F26AFF2D0110720FEF74AFDFA
:1067D00095F83700012814D197A1FEF743FD98A141
:1067E0000720FEF73FFD984B1878E864FFF7BEFFDF
:1067F00095F84C001870FFF7C9FF85F83200C5E91D
:10680000186495F83700022815D190A10120FEF7F1
:1068100029FD8BA10720FEF725FD8E4B1878E86433
:10682000FFF7A4FF95F84C001870FFF7AFFF85F84D
:106830003300C5E9186495F83700032815D186A1FF
:106840000120FEF70FFD7EA10720FEF70BFD844B14
:106850001878E864FFF78AFF95F84C001870FFF786
:1068600095FF85F83400C5E9186495F837000428C9
:1068700011D17CA10120FEF7F5FC7CA10720FEF7D9
:10688000F1FCDFF8F0C19CF80000A870FFF756FF9C
:10689000A8788CF8000095F83700052811D176A16A
:1068A0000120FEF7DFFC76A10720FEF7DBFC764B2C
:1068B0001878E864FFF75AFF95F84C001870C5E99E
:1068C000186495F83700062811D170A10120FEF751
:1068D000C9FC70A10720FEF7C5FCDFF8C0C19CF819
:1068E0000000A870FFF72AFFA8788CF8000095F840
:1068F0003700072811D16AA10120FEF7B3FC6AA175
:106900000720FEF7AFFCDFF8A8C19CF80000A870D4
:10691000FFF714FFA8788CF8000095F837000828D6
:1069200011D164A10120FEF79DFC53A10720FEF7C1
:1069300099FCDFF888C19CF80000A870FFF7FEFE04
:10694000A8788CF8000095F83700092811D15CA1CF
:106950000120FEF787FC5CA10720FEF783FCDFF82F
:1069600070C19CF80000A870FFF7E8FEA8788CF8CA
:10697000000095F837000A2819D151A10120FEF72F
:1069800071FC54A10720FEF76DFC95F82500012845
:1069900002D1A96DC8F80010D8F80000E864686555
:1069A0004FF47A704EF66021C5E91810E86595F845
:1069B00037000B2811D149A10120FEF753FC35A166
:1069C0000720FEF74FFCDFF81CC19CF80000A87000
:1069D000FFF7B4FEA8788CF8000095F837000C2873
:1069E0000CD141A10120FEF73DFC20A10720FEF7BC
:1069F00039FCDFF8FCC09CF800007BE080E0000080
:106A000036040020350400209806002040420F0084
:106A10008804002032040020A80400209C040020E8
:106A20008C040020D40200203B040020F807002042
:106A3000A0040020A608002020206C6566740000D9
:106A4000636F696E7300000029040020207269677B
:106A5000687400002A04002063656E74657200008B
:106A60002B04002020636875746500006D617463F9
:106A700068000000280400206372656469740000E7
:106A80006C696D6974000000430400202020636F6E
:106A9000696E0000736F756E647300003904002026
:106AA000202073686F7700006372656473000000D4
:106AB0003404002073706563696100002F040020B6
:106AC00073706563696C00006F76657272640000B4
:106AD0002E04002061776172640000002073636FF0
:106AE000726500003A040020656E61626C6500000A
:106AF00031040020A870FFF721FEA8788CF8000070
:106B000095F837000D2812D1FEA10120FEF7AAFB4F
:106B1000AFF294010720FEF7A5FBFC4B1878E86460
:106B2000FFF724FE95F84C0018700820286695F8A9
:106B300037000E2811D1F6A10120FEF793FBF6A134
:106B40000720FEF78FFBDFF8D8C39CF80000A87081
:106B5000FFF7F4FDA8788CF8000095F837000F28AF
:106B600012D1AFF27C010120FEF77CFBEDA10720E2
:106B7000FEF778FBDFF8B4C39CF80000A870FFF7BD
:106B8000DDFDA8788CF8000095F8370095F83810EE
:106B900088420FD1E6A10120FEF764FBE6A10720A1
:106BA000FEF760FB4FF0FF30EC65E86495F82500D8
:106BB000012819D0AFF2C0511120FEF753FBE96C48
:106BC000002902DB1620FEF70CFBDD49886C401E15
:106BD000886409D0FFF7EBF985F8250001280ED06D
:106BE000022819D003281CD0D6A10120FEF73AFBB9
:106BF000AFF2FC51BDE8F0470720FEF733BBD5E903
:106C000017010A1A696D8A4201DA686E00E00844C9
:106C1000A86589F80070D6E5686EA86585F82570C6
:106C2000F7E795F8370095F83810884202D185F8D3
:106C30003770C8E5401C85F83700C4E5C34810B577
:106C4000006880470C21BDE810400120FEF702BC1F
:106C5000BB480021803800F8281F4170B8485C30DC
:106C600002F0B5BD30B5B649B948A1F18004CA6893
:106C7000006894F83610B74B50B1884208D91D68A7
:106C8000411A6943B1FBF0F1B2FBF0F2114401E0AB
:106C900092FBF1F11960B0490A78002A2DD0AF4972
:106CA0000A28096802D8B1EB500F26D96425694338
:106CB000B1FBF0F12165881A1B686430584390FBE2
:106CC000F5F042F2107390FBF3F05843A44B984256
:106CD00000DDA448914210D0A34900EB0012A34B61
:106CE00008600A2192FBF1F21A6000EBC00202EB8D
:106CF000001090FBF1F09E49086030BD70B5904DDA
:106D00000120A5F180046861A06E6426E06490FB18
:106D1000F6F106FB1100A86194F82B10884201D10E
:106D2000FFF729FC6869401C686194F836108842B6
:106D30000AD8022804D0032804D02868E064E6E7D3
:106D4000206FFBE7A06FF9E770BD10B57C4C002009
:106D5000803CA076AFF260710120FEF783FAAFF2BB
:106D600068710720FEF77EFA0620A16EFEF739FA59
:106D700094F83600012805D9216FBDE810400C2099
:106D8000FEF72FBA16E42DE9F0476D4C803C94F8DD
:106D9000450002287DD02046E1780079002504F5E1
:106DA000AA79012601B110B9617E002972D0A07EB6
:106DB00058B163489830007802F0D0FD6048A430A4
:106DC000007802F0CBFDFFF7C0FF6A4800688047FB
:106DD000607EA0B1657602210020FEF73BFB84F8BF
:106DE0004560AFF2EC716448FDF7C0F862492C20B1
:106DF000FEF738FA60492620FEF734FA02E05F48D1
:106E00000068804799F8000002F0A8FDE57094F84A
:106E100026004B4F18B1401E84F826001AE094F863
:106E20003E0094F83610884211D15549E07E097829
:106E3000884208D2401CC1B2E1762E20FEF7D1F97B
:106E400084F83E6006E0022084F8450023E0401C00
:106E500084F83E0094F8450002281CD0207A0028CF
:106E60004ED0DFF820810620D8F80010FEF7B9F9DF
:106E700045480078002844D0444801680C20FEF7BB
:106E8000B0F9434801681620FEF7ABF941480168A4
:106E9000A9E020E1E6E001210020FEF7DBFA3E4810
:106EA0000078A8B10A207861FCF73DFC397D4843A1
:106EB000C1B284F82B102E20FEF793F994F82B0022
:106EC00018B900212D20FEF78CF9FFF717FF04E019
:106ED000AFF6D8012D20FEF7C5F9A06EF860E0648A
:106EE00094F8360001286BD0FFF79AFBF968206F01
:106EF0000144F960E06494F83600022860D04DE067
:106F000074E064E0657862616C6C00004404002009
:106F100020204853544400006177617264200000CF
:106F2000360400206164766E63650000470400202B
:106F30006F7074696F6E7300646F6E65000000009F
:106F4000180700206F7074696F6E0000A4020020A3
:106F50005804002094040020250400209004002000
:106F6000801A060070F305008404002098040020B5
:106F7000A4040020B4020020D30B0020B80200209B
:106F8000270400208C040020320400209C040020F0
:106F9000A80400208804002031040020FFF740FBF3
:106FA000F968A06F0144F960E06494F836000328A2
:106FB00006D0FFF735FBF96838680144F960E064F2
:106FC000FFF72EFBFFF74EFEFCF7CFF85AE00C2040
:106FD000D8F80010FEF705F91620D8F80010FEF7D3
:106FE00000F9D8F800101C20FEF7FBF8F8480068FC
:106FF0008047FEF7B4FAF74800688047AFF60821EB
:10700000F548FCF7B3FFF4490120FEF72BF9F249EC
:107010000720FEF727F9F0491120FEF723F9EE4982
:107020001720FEF71FF90620A16EFEF7DAF894F894
:107030003600012813D90C20216FFEF7D2F894F8FE
:10704000360002280BD91620A16FFEF7CAF894F873
:107050003600032803D91C203968FEF7C2F8FFF771
:1070600032F90FE048B9DD482671E570007802F08A
:1070700075FC04210020FEF7EDF9D948006880472F
:10708000FEF729FF94F84500022824D1D348183090
:10709000007802F063FCD1482430007802F05EFCF6
:1070A00099F8000002F05AFC04F80D6F0C21E57607
:1070B00025770120FEF7CEF9FFF7C0FD0121002062
:1070C000FEF75CFEC748007808B1FFF7C1FDBDE8D8
:1070D000F047FCF74AB8BDE8F08710B5FEF776F840
:1070E000FEF73DFA01210020FEF7B4F9BE48007812
:1070F00030B1BE4801784FF030000029FEF771F83A
:10710000B848007808B1FFF7A3FDB9480078FFF749
:107110003DFBB249E83901F8320FB6480078FFF775
:1071200035FB4870B4480078FFF730FB88700321C6
:10713000BDE810400120FEF78DB970B50546FFF798
:10714000D8FAA64CE83C607E617D08430CD1AB4880
:1071500000688047012084F8450094F83D006843AA
:10716000BDE8704000F07EB870BD70B5A4489B4D7E
:107170000078683DA5F1800468B1A2480068FFF777
:10718000DCFFA148007818B105210220FEF7F6FDCA
:10719000E07E686470BDE17E686C8842F8D09B48F0
:1071A000007810B1FFF7E7F901E0FFF734F894F841
:1071B0004000401C84F84000EAE702469448016819
:1071C00000290FDD8A420BDD92480068884209DD04
:1071D000824206DD90490968814203DD8A4201DA74
:1071E000084670470020704710B57C4C8B4AE83C3D
:1071F000116894F83E00491C012811D002281AD0C9
:10720000032823D080346368002B2ADD206898424D
:1072100027DD1160FFF7D1FF6060BDE81040A4E7F3
:10722000E36E002B1DDDA06E98421ADD1160FFF7A2
:10723000C4FFE066F1E7636F002B12DD206F984218
:107240000FDD1160FFF7B9FF6067E6E7E36F002B22
:1072500007DDA06F984204DD1160FFF7AEFFE06725
:10726000DBE78FE570B55D4DE83D2A4695F83E10A9
:10727000927E05F18004012908D002290FD003294C
:1072800016D0216801442160DAB11DE0A96E0144E5
:10729000A96612B90620FDF7A4FFA86E15E0296FB4
:1072A0000144296712B90C20FDF79BFF286F0CE001
:1072B000A96F0144A96712B91620FDF792FFA86FC4
:1072C00003E01C20FDF78DFF2068A0605448007883
:1072D00068B1A97D012009B1206108E0514AA16887
:1072E000914204DDA8753D48183002F070FABDE8FF
:1072F000704079E770B5394DE83DA87D00285FD032
:10730000484EA96E05F18004B1420CDD2069B042FF
:1073100004D1AFF61C510120FDF7A4FFA86E21692E
:1073200090FBF1F1E9640620FDF75BFF296FB142A4
:107330000CDD2069B04204D1AFF644510720FDF7BF
:1073400091FF286F216990FBF1F1E9640C20FDF7B2
:1073500048FFA96FB1420CDD2069B04204D1AFF6FD
:1073600068511120FDF77EFFA86F216990FBF1F1B4
:10737000E9641620FDF735FF2168B1420CDD206974
:10738000B04204D1AFF690511720FDF76BFF216991
:10739000206890FBF1F1E9641C20FDF722FF2069D1
:1073A000012809D00A2190FBF1F020610B48183028
:1073B000BDE8704002F00BBA084826612430F7E7B8
:1073C00070BD06490020E839C87242F21070B4E678
:1073D000A0020020AC020020D30B00208007002078
:1073E000A8020020370400203404002045040020B7
:1073F000290400202A0400202B040020CC020020B5
:107400002E040020A0040020390400202F040020B6
:107410008404002098040020A4040020900400208C
:107420003504002040420F00FE4810B590F843009C
:1074300070B1012813D0022817D0AFF2F841012013
:10744000FDF710FFF8A1BDE810400720FDF70ABFC7
:10745000F7A10120FDF706FFAFF66461F3E7F6A19F
:107460000120FDF7FFFEF6A1EDE7F7A10120FDF7F2
:10747000F9FEF7A1E7E7EB4890F82510012901D0C4
:10748000C16C01E0816DC1644165F3494166F34916
:10749000016642F21071C1657047704710B5E14C4A
:1074A000607E002843D194F8450002283FD0EC4884
:1074B0000178E1B194F844000122401CC0B284F884
:1074C000440081421CD1E7490868401C086062768C
:1074D00002210120FDF7BEFF03210220FEF74EFC32
:1074E000042084F84500BDE81040FBF73EBE0220B2
:1074F00084F845000121BDE810400020FDF7AABF37
:10750000D948A276007802F029FAD7480C300078E2
:1075100002F024FAD44802F05AF9D3480C3002F0B1
:1075200056F9BDE81040D1A10120FDF79BBE29E42A
:10753000BC4991F84400002802D0401E81F8440064
:107540007047B84900208871704710B5B54C207F4E
:107550000A280AD3142801D3E07F00E0A07F84F832
:107560002A00C1B20120FDF775FF207F0A21B0FB80
:10757000F1F201FB1200AB498031002888610AD08A
:10758000617F0844401EC1B284F82A10BDE8104053
:107590000120FDF75FBF64E610B5A24C207F1428E0
:1075A00006D01D2804D00A2804D0132802D007E0F2
:1075B000E17F14E0A17F84F82A100020FDF74AFF44
:1075C000207F0A21B0FBF1F201FB120095498031C6
:1075D000002888610AD0617F0844401EC1B284F847
:1075E0002A10BDE810400020FDF734BF39E610B581
:1075F0008C4C207F94F82D10884207D2FFF7CCFFE7
:10760000207F401C2077BDE810409EE729E670B53A
:10761000844C94F8200094F82C10884213D204F182
:10762000CC05284410F8011C11B10020FDF712FF11
:1076300094F82000295C11B10120FDF70BFF14F82C
:10764000200F401C207070BD70B5764D95F820005D
:10765000012817D905F1CC04204410F8011C11B100
:107660000020FDF7F7FE15F8200F401EC0B228706D
:10767000204410F8011C002904D0BDE8704001200E
:10768000FDF7E8BE70BD10B5664C042194F82800E3
:10769000F0B1312820D0401C84F8280094F829004B
:1076A00031281CD0401C84F8290014F8280FFDF75D
:1076B00084FF20706078FDF780FF607021780120E2
:1076C000FDF7C8FE6178BDE810400020FDF7C2BE9E
:1076D00084F828102D20E6E784F82810DEE784F8E7
:1076E0002910E2E72DE9F0414E4C0025012684F8EF
:1076F000255084F837600B20604F84F838006049CB
:107700000120FDF7AFFD5E490720FDF7ABFD94F8C2
:10771000370001280AD15BA1FDF7A4FDAFF678413F
:107720000720FDF79FFD59480078E06494F8370082
:1077300002280AD156A10120FDF794FD56A1072089
:10774000FDF790FD56480068E06494F83700032880
:107750000AD154A10120FDF785FD54A10720FDF7B2
:1077600081FD54480068E06494F8370004280BD188
:107770004CA10120FDF776FDAFF624510720FDF75F
:1077800071FD4D480068E06494F8370005280AD17F
:1077900044A10120FDF766FD48A10720FDF762FD29
:1077A00048480068E06494F8370006280AD135A1FB
:1077B0000120FDF757FD44A10720FDF753FD444884
:1077C0000068E06494F8370007280AD141A101203D
:1077D000FDF748FD41A10720FDF744FD4148006841
:1077E000E06494F8370008280AD13AA10120FDF797
:1077F00039FD3DA10720FDF735FD3D480068E064F7
:1078000094F8370009280AD132A10120FDF72AFD9A
:1078100038A10720FDF726FD12480068E06494F8BF
:1078200037006BE0980600207365747570000000E7
:1078300020646F6E652000002067616D65000000A8
:107840007374617473000000686172647772000081
:10785000746573747300000080380100301B0F00E2
:107860004604002074040020B007002077686F6190
:1078700068206275626261200000000094040020AC
:10788000F865000820746F74616C000045040020E6
:10789000202067616D65000073746172747300006D
:1078A0005804002020636F696E730000206C6566C9
:1078B000740000005C0400206404002072696768A2
:1078C00074000000600400207265706C6173000039
:1078D000700400206E756D6265720000736C616DDE
:1078E000730000006C0400206562616C6C73000022
:1078F0006804002074696C74730000000A280ED1BB
:10790000FCA10120FDF7AEFCFCA10720FDF7AAFCBD
:107910003868E06494F82500022800D13D6094F8AE
:10792000370094F83810884210D1F6A10120FDF7F5
:1079300099FCAFF6FC110720FDF794FC4FF0FF30E7
:10794000E565E06494F82500012818D0EF4911207E
:10795000FDF788FCE16C002902DB1620FDF741FCF5
:10796000EB48816C491E8164FEF721FB84F82500F9
:1079700001283FF4C4AE022807D003280AD0BDE88E
:10798000F041E2490720FDF76DBC606EA06584F808
:107990002560B4E694F8370094F83810884202D194
:1079A00084F83760ABE6401C84F83700A7E6D84877
:1079B000D849803890F83E00022801D8112000E014
:1079C0000120FDF74FBC10B5D14CD049803C94F854
:1079D0003E00022816D81120FDF744FCCB491720A1
:1079E000FDF740FC94F83E00022803D91620A16F51
:1079F000FDF7F7FB94F83E00032818D9C448016846
:107A00001C2010E00120FDF72DFCC0490720FDF7E8
:107A100029FC0620A16EFDF7E4FB94F83E00012846
:107A200005D9216F0C20BDE81040FDF7DABB18E442
:107A300010B5B9A10120FDF715FCB948007808B1CF
:107A4000B8A100E0B9A10720FDF70CFCB04C803CC8
:107A500094F82700E0B1B7A11120FDF703FCAB4972
:107A60001720FDF7FFFB94F8270098B1012813D0E9
:107A7000B24801681C20FDF7B4FB14F8270F401C26
:107A8000C0B20321B0FBF1F201FB120020704EE501
:107A9000ABA1E1E7AC48ECE7AC48EAE770B5AC4C29
:107AA000AC4E9B4D2068B04244DD2869B04213D1F2
:107AB00096499848FCF75AFA96490120FDF7D2FBFF
:107AC00094490720FDF7CEFB92491120FDF7CAFB30
:107AD00090491720FDF7C6FB206829698C4C90FB64
:107AE000F1F1803C0620E164FDF77BFB9A480078C9
:107AF00068B39A480168B14203DD286991FBF0F14F
:107B0000E1640C20FDF76DFB95480168B14203DD8F
:107B1000286991FBF0F1E1641620FDF762FB9148C2
:107B20000168B14203DD286991FBF0F1E1641C209A
:107B3000FDF757FB2869012813D00A2190FBF1F0CB
:107B40002861BDE870407248743001F040BE0C20DE
:107B5000E16CFDF746FB1620E16CFDF742FBE16CA2
:107B6000E5E72E61EDE72DE9F047694C803CA07B0D
:107B700000287CD165496748FCF7F8F994F845007E
:107B80000027DFF8D0910125614E022810D0E1785E
:107B900000296CD104286AD0A079A17D084366D160
:107BA000607B00287AD06773A07E002877D019E127
:107BB000A07900285BD16C480078002857D055493F
:107BC0000120FDF74FFB53490720FDF74BFB5149BF
:107BD0001120FDF747FBDFF8948198F8000018B9F1
:107BE0004C491720FDF73EFB49487430007801F0FE
:107BF000B5FE47488030007801F0B0FE44488C3034
:107C0000007801F0ABFE607BDFF864A1F8B1677328
:107C10000B210020FDF71EFC9AF8000030B1A07D7A
:107C200020B1C6F81090FFF765FB5FE00620A16E5B
:107C3000FDF7D7FA0C20216FFDF7D3FA1620A16FBC
:107C4000FDF7CFFA98F8000038BB31684BE049489F
:107C50006573007888B1A57094F82300401CC0B209
:107C600084F82300022809D984F8277000E0BFE0D7
:107C7000FFF7DEFE84F8237038E0A7700B210120A7
:107C8000FDF7E8FB9AF80000314F48B139684945E3
:107C900006DDC6F81090FFF701FF27E085E06BE0F6
:107CA00006203968FDF79DFA2B48007878B12B48FB
:107CB00001680C20FDF795FA294801681620FDF7A8
:107CC00090FA98F8000088B9264801680BE00C206B
:107CD0003968FDF786FA16203968FDF782FA98F8B8
:107CE000000018B939681C20FDF77BFA0848A57117
:107CF000B03079E0617665726167000073636F721E
:107D0000652000002020646174610000F8650008AF
:107D100018070020D30B00202065787472610000E2
:107D20002F04002067616D652020000062616C6C8B
:107D300020200000616E642061740000A404002013
:107D4000202061742020000084040020980400207A
:107D50008C04002040420F00320400209C040020CC
:107D6000A804002088040020330400203C040020E4
:107D7000350400202504002094F83E00012806D098
:107D8000022807D0032808D004282BD108E0FA499C
:107D9000012007E0F849072004E0F749112001E03D
:107DA000F5491720FDF75EFA1CE06573C6F81090E0
:107DB000A07EB8B994F83E00012806D0022807D06A
:107DC000032808D004280DD108E00620A16E07E0A2
:107DD0000C20216F04E01620A16F01E01C20316807
:107DE000FDF7FFF9E548A571BDE8F04701F0EFBCEC
:107DF000BDE8F0872DE9F05FE14D0024012685F80C
:107E00002540E04FDFF88093DFF880A3DFF8808320
:107E1000DFF880B385F82E60DF490720FDF722FAEE
:107E200095F82E00012811D1AFF25851FDF71AFA3A
:107E3000DAA10720FDF716FADA4B1878E864FEF7A6
:107E400095FC95F84C0018700820286695F82E00CF
:107E500002280ED1D4A10120FDF704FAD4A10720F5
:107E6000FDF700FAD44A1068E864FFF704FBE86CF9
:107E7000106095F82E0003280ED1D0A10120FDF747
:107E8000F1F9CBA10720FDF7EDF9CE4A1068E864BF
:107E9000FFF7F1FAE86C106095F82E0004280ED177
:107EA000C9A10120FDF7DEF9C1A10720FDF7DAF92C
:107EB000C74A1068E864FFF7DEFAE86C106095F8CE
:107EC0002E00052810D1C3A10120FDF7CBF9AFF298
:107ED000D4110720FDF7C6F9D8F800004246E8643F
:107EE000FFF7C9FAE86C106095F82E00062812D149
:107EF000BAA10120FDF7B6F9BAA10720FDF7B2F942
:107F0000BA4B1878E864FEF731FC95F84C0018700D
:107F10001E20C5E9180495F82E00072812D1B4A137
:107F20000120FDF79FF9B4A10720FDF79BF9B44BA1
:107F30001878E864FEF71AFC95F84C0018702820B1
:107F4000C5E9180495F82E00082811D1AD49012083
:107F5000FDF788F9ACA10720FDF784F9DFF8B0C27E
:107F60009CF80000A870FEF7E9FBA8788CF80000E8
:107F700095F82E00092812D1A24901204839FDF7B1
:107F800071F9A4A10720FDF76DF9DFF890C29CF804
:107F90000000A870FEF7D2FBA8788CF8000095F8D6
:107FA0002E000A2823D197490120FDF75BF99CA1F7
:107FB0000720FDF757F93878A870FEF7BFFB38782F
:107FC000012812D1A87880B9974AD8F800109142B8
:107FD0000BDD9649C8F800109549C9F8001095497D
:107FE000CAF800109449CBF80010A878387095F8BA
:107FF0002E000B2813D1AFF274710120FDF732F976
:108000008EA10720FDF72EF98E4B1878E864FEF755
:10801000ADFB95F84C0018700520C5E9180495F8DB
:108020002E000C2811D188A10120FDF71BF988A191
:108030000720FDF717F9DFF820C29CF80000A870B0
:10804000FEF77CFBA8788CF8000095F82E000D2830
:1080500011D182A10120FDF705F982A10720FDF7CA
:1080600001F9DFF808C29CF80000A870FEF766FB73
:10807000A8788CF8000095F82E000E2811D17CA16C
:108080000120FDF7EFF87CA10720FDF7EBF8DFF802
:10809000F0C19CF80000A870FEF750FBA8788CF89F
:1080A000000095F82E0095F83010884206D395F818
:1080B0002F10884202D273480068804795F82E003E
:1080C00095F82F1088420FD16FA10120FDF7CAF853
:1080D0006FA10720FDF7C6F84FF0FF30EC65E864AC
:1080E00095F8250001281AD02B491120FDF7BAF880
:1080F000E96C002902DB1620FDF773F82049803176
:10810000886C401E88640CD0FDF7B1FF95F82500FF
:10811000012810D002282AD0032829D001E085F8B0
:108120002E6059A10120FDF79DF8BDE8F05F1A49C6
:108130000720FDF797B8D5E91710421A686D8242FB
:1081400001DA686E00E00844A86595F82E0005285D
:108150000FD1A86D90FBF1F0484344F62061C8F8B8
:108160000000884206DD411AC9F8001096E0ACE034
:10817000B0E0A7E090E00000D30B0020D40700207F
:1081800098060020350400209C040020A80400204C
:108190008C04002088040020F865000862616C6C83
:1081A00073000000270400202066697273740000C9
:1081B0007468726573680000840400207365636FDF
:1081C0006E640000980400202074686972640000E6
:1081D000A4040020202068696768000020206175E1
:1081E000746F000070657263656E000025040020E6
:1081F000202062616C6C00007361766520200000B5
:1082000026040020E86A0008342048535444000043
:1082100032040020687374642020000033040020BE
:108220006D696C696F6E000040420F00E0E60B0064
:1082300020120A00603D0800A068060074696C7492
:1082400073200000460400202069646C6520000053
:10825000616E696D617400003704002020666173EF
:1082600074200000626F6E757320000030040020DF
:1082700020736B696C6C000073686F7420200000C1
:108280003B040020C4020020207365747570000058
:10829000646F6E6520200000C9F8004047F230513D
:1082A000884203DD411ACAF8001001E0CAF8004014
:1082B00049F64041884203DD401ACBF8000001E056
:1082C000CBF80040FC480670A6E5686EA86585F806
:1082D0002560F7E795F82E0095F82F10884202D117
:1082E00085F82E6098E5401C85F82E0094E5F3494A
:1082F00010B50868F24C401C0860F24814F8321FB0
:108300000078FEF7CAF92070ED4C803401E0FDF7EB
:108310005FFF6069401E6061401CF8D110BDEA49F2
:1083200010B50868E64C401C0860E84814F8341F93
:108330000078FEF7B2F92070E14C803401E0FDF7DF
:1083400047FF6069401E6061401CF8D110BD704756
:1083500070B500240D46224608E0295D04F10104B1
:10836000E4B20029F9D102F10102D2B28242F4D37F
:1083700004E0641CE4B20620FDF76CF8295D0029D6
:10838000F7D170BDFDF7DFBF10B5CD4CE07B002805
:1083900005D0FDF7E4F8FDF787F90020E07310BD84
:1083A000CB4810B50168C64C491C0160C94800782B
:1083B00018B114F8321FC34802E014F8331FC6483E
:1083C0000078FEF76AF92070BD4C803401E0FDF7BB
:1083D000FFFE6069401E6061401CF8D110BDB84AC4
:1083E000012802F1800105D0022805D0032806D01B
:1083F000086802E0906E00E0106F88607047906F30
:10840000FBE72DE9F0410446AD481746884690F851
:108410003E00FFF7E4FFAA4D80356426A86012E015
:10842000A86890FBF6F106FB110068610A20FEF7D0
:1084300084FE68695A280BD041460020FDF79EFC57
:10844000A8680A30A860641EE4B2E9D2BDE8F081F1
:108450003946F2E72DE9F0470446994890468946A7
:1084600090F83E00FFF7BBFF954D4FF47A768035CC
:108470004FF46177A86014E0A86890FBF6F106FB62
:10848000110068616420FEF758FE6869B84201D1A6
:10849000414600E049460020FDF770FCA8686430C2
:1084A000A860641EE4B2E7D2A2E42DE9F0410F46D1
:1084B00004464FF47A76894D09E03046FEF73DFEDA
:1084C00039460020FDF75AFC286801F00AF8641EBE
:1084D000E4B2F2D2BAE72DE9F041794C804D7F4FFA
:1084E000E0794FF47A7690B3207F84F8410094F8D5
:1084F000201004F1CC00084410F8011C0120FCF706
:10850000A9FF1FE094F841000FE0FFF71EF8304686
:10851000FEF713FE61780020FDF730FC286800F0BC
:10852000E0FFFFF739F8207F401E207710F0FF0FA3
:10853000EBD1386800F0D5FF94F82000012807D966
:10854000FFF782F894F820000028DBD17EE722E0D4
:10855000002084F8200079E7FEF7F7FF94F8200068
:108560000CE03046FEF7E9FD61780020FDF706FCDF
:10857000286800F0B6FF94F84100401E84F84100DE
:1085800010F0FF0FEDD1FFF707F8207F401E207796
:10859000386800F0A6FF207F0028DDD156E770473D
:1085A000504810B50168491C01604549022081F816
:1085B000450001210020FCF74DFF02210120FCF7BE
:1085C00049FFFCF703FEFDF786FC47A10120FCF7FD
:1085D00049FE47A10720FCF745FE00F0A0FF01F08F
:1085E00042F845490020086003210220FDF7C6FB40
:1085F000FAF7BBFD41F2883000F052FF3F480068B7
:10860000BDE81040004710B58AB006281AD2DFE84E
:1086100000F019030D29333D39A10120FCF722FE9A
:1086200039A10720FCF71EFE39A108E03DA1012079
:10863000FCF718FE3DA10720FCF714FE3DA168469B
:10864000FBF794FC40480078032802D36846FBF708
:1086500012FC1B4C8020012184F845000020FCF70F
:10866000F9FE1FE039A10120FCF7FCFD2FA1072036
:10867000FCF7F8FD37A1E2E73BA10120FCF7F2FD92
:108680002AA10720FCF7EEFD39A1D8E73DA1012082
:10869000FCF7E8FD25A10720FCF7E4FD3BA1CEE7B0
:1086A000FDF719FCFDF732FC7028F9D1022084F89F
:1086B00045000AB010BD0000A60800205C040020A0
:1086C0009806002029040020640400202B040020C8
:1086D00060040020280400202A0400205004002008
:1086E0004C0400206C040020202062616420000003
:1086F000206F6E652020000034090020A4020020B5
:1087000073776974636800006F7672666C6F00003F
:108710005377697463682051204F766572666C6F79
:10872000770000007174696D65720000777463688A
:108730006467000054696D6572205461626C652045
:1087400066756C6C00000000D003002071657665D2
:108750006E7400004576656E74205461626C65200D
:1087600066756C6C00000000636576656E740000D1
:10877000436F756C646E7420636C656172206576FE
:10878000656E7400756576656E740000436F756C78
:10879000646E74207570646174652074696D6572AF
:1087A0000000000010B5D14C4FF00B01A07808B1CB
:1087B000012000E00020FCF74DFEA07810B1002061
:1087C000A07077E70120FBE7C848417C11B1002188
:1087D0004174704701214174C5480068004710B5D5
:1087E000142839D2DFE800F0380A0D1113161A1DCB
:1087F0002020232629292D3033353B3BFDF762FE0F
:108800002DE0BC480068804729E0BB4803E0FFF743
:10881000BBFD24E0B9480068804720E0FDF768FE12
:108820001DE0FFF73BF91AE0FEF764FD17E0FEF7E5
:108830007FFE14E0FEF789FA11E0AC490020887150
:108840000DE0FFF7C1FF0AE0FDF77DFD07E0AC4852
:10885000E1E7FFF7A7FF02E0AA490968884700207F
:1088600028E710B5703808281ED2DFE800F00407AA
:108870000A0D1013161900F01BFD13E0FFF737FD6A
:1088800010E0FFF78DFD0DE0FFF749FD0AE0FDF771
:108890005AFD07E0FEF702FE04E0FEF774FA01E07D
:1088A000FFF77EFE002005E74FF0FF3002E770B5CE
:1088B0009548002497490470944801250470944811
:1088C00004700520087094489AA1057093480460CC
:1088D000934804609348046093480570934805707A
:1088E000934805709A48FBF741FB9A489D49B74A5F
:1088F00004709948BB4B04709848057098480570FF
:1089000040F6C410086098489A490470974804706B
:108910009748086099499848086099489A490460BE
:108920009848086099489C4905709948057099488D
:1089300005700F2008709948994904700320087049
:1089400098490C7098490C6098490C6098490C60E3
:1089500098490C6098490C6098490D7098490C60D2
:1089600098490D70984911609A4A994911609A4A3C
:1089700014709A4A14709A4A157044F620621A606C
:10898000994A1470994B4FF47A721A60984BC82226
:108990001A70984A1160994A97491160984908706D
:1089A00098494620086098495F200860974899498F
:1089B000047097480470642008609749DC200860C0
:1089C00070BDF0B595480123954906780020954A79
:1089D000954C964D0C2E11D2DFE806F010061113BF
:1089E000061511091310191D0870107005E0904943
:1089F000122008708F49087032202070F0BD287056
:108A0000F0BD0B7005E0087028702370F0BD287071
:108A100008701370F0BD0870F0BD2DE9F041334CC3
:108A2000324F0126803704F8026F00257D61BD6159
:108A3000C4F84A50C4F84E507FA181481E34FBF759
:108A400095FA04F81D5C04F81A5C4FF00F0804F85E
:108A5000038C66700A20A07004F8195C6563E570E9
:108A60002571A563657104F8165C022084F8250061
:108A700004F8145C04F8136C04F8125C6EA107F19E
:108A80005100E563FBF772FA7D6225726572A5728B
:108A900004F8115C84F80D802564A67384F81080B6
:108AA00065646574A674E674267584F81580E675A9
:108AB00084F818804FF44870B86240103862FA2089
:108AC000F862E5775FA1A7F13A00FBF74FFAFD6086
:108AD00004F8105C04F80E5C04F80B5C84F8225077
:108AE0004FF41670B86404F8155CAFE498060020E3
:108AF000D0020020A4020020C8020020BC020020F6
:108B0000D402002088020020240400202504002034
:108B10002604002027040020280400205C040020F4
:108B20006004002064040020290400202A0400209E
:108B30002B04002053797374656D383020435055F1
:108B4000202041524D20206D6F64656C00000000B4
:108B5000430B00202C0400203204002033040020AA
:108B60003404002054040020350400204704002071
:108B7000C0D4010084040020708203008804002017
:108B80005804002000E204008C0400203604002079
:108B90003704002031040020420400204304002058
:108BA0004404002045040020680400206C040020D8
:108BB0007004002090040020740400203904002078
:108BC000940400203A04002020BF020098040020F2
:108BD000C04504009C0400203B0400202E0400201B
:108BE0002F040020A004002030040020780400207E
:108BF0002D040020A404002090D00300A80400202D
:108C0000460400204C040020500400203C040020B6
:108C10003D0400207C040020800400204804002043
:108C200020040020210400203F0400203E040020F6
:108C300040040020410400206E756C6C00000000B0
:108C4000D30B0020312E32360000000010B5FDF7A6
:108C50006FF9FF280AD0FDF76BF9702808D0742847
:108C600006D0FDF753F9FF4900200870002010BD21
:108C7000012010BD2DE9F041FB4FFC4D4FF49678DB
:108C8000C7F800802878012405F13306002871D048
:108C9000C0EBC00081190720C91FFCF7E3FA27E0E9
:108CA000FDF785F9012804D0022852D003281FD1EE
:108CB00053E0EC49002008702878072818D2DFE834
:108CC00000F048040C0F1215220024B100242046A5
:108CD000FCF709FB0CE00124F9E7FCF7F5FC07E0E1
:108CE000FCF7B9FF04E0FDF7DBF901E0FDF76CF8F4
:108CF0003868401E3860401CD2D1DD49022008701F
:108D00000120BDE8F081FFF7D2FDDA48DA4A0068B9
:108D1000A0F59C4120391160D84AA0F5EA413039CC
:108D20001160D749A0F51C404038086001206870E8
:108D300003210020FCF744FFCC490720891CFCF7E5
:108D400091FA4FF4FA7000F0CCFBC8494F3107207C
:108D5000A3E7FCF73BFA0020D3E7C7F800802878A8
:108D600001240721401CB0FBF1F201FB1200287026
:108D70008CE7FFE7BD49891C07208EE72DE9F0410C
:108D8000B94C4FF49670BF4D2060BFA12F780720DB
:108D9000FCF768FADFF8F8822978112058F82110DA
:108DA000FCF760FA002640E0FDF701F9012804D045
:108DB000022812D0032838D112E0B6480C210670E0
:108DC0002878401CB0FBF1F201FB1200287058F823
:108DD00020101120FCF746FA27E02E70002090E7C3
:108DE000ADA10720FCF73EFAABA11720FCF73AFA39
:108DF0002878B84218D09D4901204870FAF729F91F
:108E000090B9A748008881B2A648007800F0F6FD26
:108E1000A548008881B2A548007800F0EFFDFFF773
:108E2000D0FDA3480068804726602068401E20606F
:108E3000401CB9D1012064E72DE9F05F01249D4970
:108E400000209D4DDFF874829D4E9E4F4FF00C0A1E
:108E5000A146087090A10720FCF704FA012C49D024
:108E6000022C52D0032C69D0042C7DD0052C7CD050
:108E7000062C7BD0072C7AD0082C79D0092C78D0FE
:108E80000A2C77D00B2C76D0544510D18EA101201E
:108E9000FCF7E8F98EA10720FCF7E4F94FF0FF306A
:108EA00028600020306083480078012818D07AA11B
:108EB0001120FCF7D7F92968002902DB1620FCF7FE
:108EC00090F969490868401E086009D0FDF7CFF89D
:108ED0007849087801287DD002287CD003287BD0EF
:108EE00079A10120FCF7BEF9BDE8F05F6AA1072077
:108EF000FCF7B8B978A10120FCF7B4F978A10720F4
:108F0000FCF7B0F9DFF8E0B109E078A10120FCF747
:108F1000A9F973A10720FCF7A5F9DFF8D8B1DBF8B0
:108F200000002860FDF722FC29681E20CBF8001005
:108F30003860A020C8F8000005203AE16EA10120A9
:108F4000FCF790F96EA10720FCF78CF9DFF8B8B1B7
:108F50009BF800002860FDF709FC28788BF80000DA
:108F600064204FF4967107E00AE022E040E061E0FF
:108F7000F2E005E11FE133E13860C8F80010DBE7FB
:108F800062A10120FCF76EF962A10720FCF76AF9E3
:108F9000DFF888B19BF800002860FDF7E7FB287830
:108FA0008BF800000A20322138600120C8F8001038
:108FB000FFE05BA10120FCF755F95BA10720FCF75E
:108FC00051F9DFF86CB1DBF800002860FDF7CEFB4B
:108FD000296802E04EE15CE163E1CBF800104FF458
:108FE0002F70386040F2DC516420C8F80010E0E0D7
:108FF00050A10120FCF736F94BA10720FCF732F90C
:10900000DFF8A4B0DBF800002860FDF7AFFB2868AC
:10901000CBF8000081B22548007800F0EFFC214930
:109020009BF800000870C820410038601420C8F880
:109030000010BEE041A10120FCF714F93AA107207D
:10904000FCF710F9DFF858B0DBF800002860FDF7F6
:109050008DFB2868CBF8000081B21248007800F040
:10906000CDFC6FE02C09002030090020A50800206D
:10907000DD0600208C0400209C040020A8040020B1
:10908000880400204804002073656C656374000048
:109090003808002024040020202020202020000068
:1090A0007C0400207407002080040020EC070020CE
:1090B0008C020020BD060020E4060020F8060020F7
:1090C000F4060020FC0600206578706572740000CC
:1090D000646F6E65202000002073636F726500006E
:1090E0006C616720746D00005004002020626F6E78
:1090F000757300004C0400202020636F696C000031
:10910000686C6420746D00002D04002020206C61C8
:109110006D700000656E6120746D000042040020D7
:10912000737769746368000073747220746D000053
:1091300078040020666C61736867000070662061C7
:109140006E690000AD489BF8001001705020386037
:10915000C820C8F800002BE0A9A10120FCF782F884
:10916000A9A10720FCF77EF8A948DFF8A8B201788A
:109170008BF80010FDF7E2FA9BF80010A4482DE0F0
:10918000AFF264010120FCF76DF8A3A10720FCF702
:1091900069F8DFF88CB29BF800002860FDF7E6FA6A
:1091A00028788BF800001E2096213860C8F800103F
:1091B0000A2030607BE69BA10120FCF753F89BA1BD
:1091C0000720FCF74FF89B48DFF848B201788BF88E
:1091D0000010FDF7B3FA9BF800109648017066E6A0
:1091E00095A10120FCF73EF895A10720FCF73AF87D
:1091F000DFF820B25FEA09008BF800901BD092A143
:109200001120FCF72FF8DFF848920DE00B21012028
:10921000FCF720F9642000F064F90B210020FCF732
:1092200019F9642000F05DF98A48D9F80010006847
:109230008142EBD019E088A11120FCF713F888488F
:1092400000F0C5FADFF8089205E0864800780228A9
:1092500001D100F000FB7F48D9F80010006881427E
:10926000F3D07F48007800F079FBFDF767FA9BF8B0
:1092700000901CE6D8F8001030680A1A7A4909688C
:109280008A4201DA386800E0084478490860012021
:1092900004E0764A3868106001200870744948700C
:1092A000D8E5544501D10124D4E5641CE4B2D1E5EC
:1092B0002DE9F05FDFF8BCB1202100208BF8001011
:1092C0000121FCF7C7F8FBF781FFFCF704FE00F073
:1092D000CAF969494FF00009DFF894A1C1F800907C
:1092E00001218AF800100D464FF416780AF10206A3
:1092F0008AF801904446F11D44E0FCF758FE01282D
:1093000004D002282DD003283FD12CE0C5EBC500A6
:1093100081190F460120FBF7A5FF072D16D2DFE8C4
:1093200005F02004070A0D101300FEF763FD0DE0A1
:10933000FEF7D8F90AE0FFF79DFC07E0FDF732FAE7
:1093400004E0FFF71BFD01E0FFF776FD002C08DDD0
:10935000444639460120FBF785FFAFF2C4211120B6
:1093600011E0002411E045486D1C44460078EDB240
:1093700008B1072000E00620A84200D10025C5EB77
:10938000C50081190120FBF76DFF201EA4F1010427
:10939000B3DC9AF80100544658B139A10120FBF71B
:1093A00061FF39A10720FBF75DFFF9F7DEFE84F8C6
:1093B00001904FF4487000F094F802255C468BF859
:1093C0000050FBF703FF3248007828B1314801789C
:1093D0003020FBF706FF04E0AFF240312F20FBF70F
:1093E00041FF2D4801782E20FBF7FBFE2B4925700D
:1093F00081F80090BDE8F05FFDF76FBE74070020B4
:10940000656E61626C65000054646562756700009A
:109410003C0400209A06002064757020746D0000E2
:109420003408002064697361626C000020536C6131
:109430006D2000003D040020202054696D6500006F
:1094400063616C69627200002077616974200000BA
:10945000700600207406002020636F7265200000F3
:1094600028080020CF030020EC060020F006002092
:10947000A5080020DD060020340900204704002054
:10948000736176696E6700006E7672616D20000010
:109490003404002045040020310400209E060020F2
:1094A00001B582B00020FE4908700120019012E051
:1094B0000120009007E0FA48007808B101980EBD3D
:1094C0000098401C009040F6782100988842F2D91C
:1094D0000198401C0190DDE901018842E8D9002093
:1094E000EDE701B583B00120029013E00120019067
:1094F00008E0EB48007810B140F624600090019835
:10950000401C019040F6782101988842F1D90298D8
:10951000401C0290DDE902018842E7D90FBD00201E
:10952000E0490880E0490870E0490870E0490870A7
:1095300040F26D10DF4908800420DF490870704751
:10954000DD480078DD4908700520DB490870704768
:10955000DA480078D849087070474188D14A1180AC
:109560008179D14A11704179D04A11700179D04A7C
:1095700011700188CF4A1180D14AC168116003215E
:10958000CD4A11707047CF480088CF490880CF4836
:1095900000780871CE4800784871CE48007888710C
:1095A000CD4800884880704700B50346FFF7EBFFC1
:1095B000C54840881844801E82B24FF47A7092FBEE
:1095C000F0F100FB1120C04948804FF47A7092FB03
:1095D000F0F082B2002A34DD08468079104482B26D
:1095E0003C2092FBF0F100FB1120B74988713C2030
:1095F00092FBF0F082B2002A23DD08464079104445
:1096000082B23C2092FBF0F100FB1120AE49487180
:109610003C2092FBF0F082B2002A12DD084600796D
:10962000104482B2182092FBF0F100FB1120A649F1
:109630000871182092FBF0F082B2084600881044AE
:10964000088000BD9B4800889F49088098480078A2
:10965000087196480078487193480078887191485D
:10966000008848807047002008E0002100EB40029D
:109670009A4B03EBC2021172411CC8B22028F4DBE2
:109680000021974A11607047014611B94FF0FF3031
:10969000704708888B4B1B88181A924B00FB03F20B
:1096A00008798A4B1B78181A4FF4616303FB002278
:1096B0004879874B1B78181A3C2303FB00228879D2
:1096C000844B1B78181A02444888834B1B889842A5
:1096D00000DD521E802A02DD4FF0FF30D8E710B2C5
:1096E000D6E7024602B111B96FF002007047108848
:1096F0000B88984201DD0120F8E710880B8898421A
:1097000002DA4FF0FF30F1E710790B79984201DD72
:109710000120EBE710790B79984202DA4FF0FF3025
:10972000E4E750794B79984201DD0120DEE750797A
:109730004B79984202DA4FF0FF30D7E790798B7976
:10974000984201DD0120D1E790798B79984202DAC5
:109750004FF0FF30CAE750884B88984201DD012066
:10976000C4E750884B88984202DA4FF0FF30BDE7DB
:109770000020BBE72DE9F041044600275848056862
:1097800001E02E466D6929462046FFF7AAFF002812
:1097900004DD3846791CCFB2FA28F2DBFA2F02DB5F
:1097A0000220FEF730FF4E480068854202D04C4848
:1097B000006840B94A480068606149480460006830
:1097C000FFF7CBFE01E074616561BDE8F0812DE932
:1097D000F04104460027A0880A2802DA781EBDE876
:1097E000F081002601E0701CC6B2202E0BDA06EBD9
:1097F00046003A4901EBC000007A20B13846791C96
:10980000CFB2FA28EFDBFA2F02DB0320FEF7FBFED4
:10981000202E02D14FF0FF30E1E706EB46002F4942
:1098200001EBC005A088FFF7BFFE2748016829604B
:109830008188A9808079A871A08828826078687260
:10984000A078E87120782872A068E8602846FFF7C1
:1098500091FF0020C3E710B54FF0FF30224909689F
:1098600008601F480068002860D01D4800681F4934
:1098700008600846006840691949086006200E49DA
:1098800008701A490968487AFEF7A9FF1748006866
:10989000C07901282CD1002014490968087245E0DC
:1098A0002C090020180900201A0900201B0900209B
:1098B0001C0900201E090020CF0300203C090020C5
:1098C000440900200E090020640F00200C0900202C
:1098D0000B0900200A09002008090020640C002060
:1098E0003409002080510100240900204009002093
:1098F00054480068C079002806DD52480068C079E5
:10990000401E50490968C8714E490968088AFFF726
:109910004BFE4C4800684C490A6802608A88828085
:109920008979817147480068FFF724FF474800683C
:1099300018B90420464908700CE0444800684149C1
:109940000968884203D041480068FFF706FE0320FB
:109950003F49087000203B49086010BD2DE9F047E1
:1099600005464FF00009C8463648006840B1354802
:109970000068007AA84203D1012032490968C87101
:109980003248006810B94846BDE8F0872F4804689F
:10999000274616E0207AA84201D0264610E04FF074
:1099A00001092A480068A04206D10620284908700B
:1099B00026496069086001E06069706100202072DA
:1099C00064692CB14046411C01F0FF086428E1DBCA
:1099D000B8F1640F02DB0420FEF715FE1B48006897
:1099E000B84204D019480068FFF7B7FD04E01748F3
:1099F000006808B9FFF793FD4846C5E72DE9F04137
:109A000005460E464FF0000800271048006810B9C0
:109A10004046BDE8F0810D48046806E0207AA8427F
:109A200002D14FF001082682646924B13846791CBE
:109A3000CFB2FA28F2DBFA2F02DB0520FEF7E3FDB6
:109A40004046E6E740090020640F0020340900206A
:049A5000CF03002020
